:100000000EC028C040C026C025C024C023C022C0C6
:1000100021C03AC01FC01EC01DC01CC01BC011247F
:100020001FBECFE5D2E0DEBFCDBF10E0A0E6B0E05E
:10003000E8EDF1E002C005900D92AE36B107D9F7B8
:1000400020E0AEE6B0E001C01D92A537B207E1F7AF
:1000500083D0C0C0D5CF0F931F9300E010E098016C
:10006000061717072807390759F0E7E8F3E1319732
:10007000F1F700C000000F5F1F4F2F4F3F4FF0CF31
:100080001F910F91089518951F920F920FB60F921E
:1000900011248F9381E080936E008F910F900FBE9B
:1000A0000F901F90189585B7806285BF1FBC88B7D9
:1000B000846088BF89B7806289BF10926E00BB9848
:1000C000C39A1FBC88958FB590916E0091118FEFE8
:1000D00099B79F7D99BFC398BB9A869508951F9342
:1000E000CF93DF9310E4C0E0D0E0DDDFC80FD11D77
:1000F0001150D9F7CE01DF91CF911F910895769BD2
:10010000FECF8FB980E48EB90895F9DF80E090E0EA
:1001100008958A3010F4805D01C0895CF0CFCF93E0
:10012000C82F82958F70F5DF8C2F8F70CF91F1CF14
:10013000CF93C82F892FF3DF8C2FCF91F0CF87B3C8
:100140008A7F87BBB99A88E18DB980E690E0909369
:100150007200809371000895F894BC9A80E886BD7F
:1001600016BC96E097BD81BFEADFC398BB9A85B7FE
:100170008F7B85BF82E080BF85B7877E85BF8BB7C9
:1001800080628BBFAB9A8FEF8BBD8EBD7894A7DF5B
:1001900000E010E0CFEFDFEFA2DF8C179D0740F00B
:1001A000C817D90730F4202F2F7319F4219601C0F6
:1001B000EC018C1B9D0B0F5F112319F0C09738F0D9
:1001C00003C08137910518F0C49A11E0E5CFC498B7
:0801D00010E0E2CFF894FFCF2C
:0E01D800000000020000000085000000000092
:00000001FF
